:100000000C9499010C94B6010C94B6010C94B601B1
:100010000C94B6010C94B6010C94B6010C94B60184
:100020000C94B6010C94B6010C94B6010C94B60174
:100030000C94B6010C94B6010C94CD020C94B6014C
:100040000C94B6010C94B6010C94B6010C94B60154
:100050000C94B6010C94B6010C94B6010C94B60144
:100060000C94B6010C94B6012C003A00456E644F16
:1000700066536F61702100312E310054616B7467DB
:100080006562657220005368757444005A75726326
:100090006B0020202020202000205368757444002D
:1000A00020004572726F72005368757464004E6F61
:1000B000726D6C0050725365300050725075420082
:1000C0002020202020202020202020002020202050
:1000D0002020202020202050726F6772004572720D
:1000E0006F720053687574640050726F6772004ECF
:1000F0006D5A5A74004E6D415A74004E6D535A74C5
:10010000004E6D566B7A004E6D537672004E6D55F3
:1001100068720020202020202000204E6F726D6C1D
:1001200000200050726F6772004E6F726D6C00207D
:100130002020002D0044002D0047002D0045002DFB
:10014000002D002D002D0045002D005379735374B0
:10015000617475732020496E69742000456E746562
:10016000722068696C66742100312E310054616B15
:10017000746765626572200055702F446F776E203A
:100180002020205A7572636B002020202020204EF2
:100190006D5A5A740055702F446F776E20202020BE
:1001A0005A7572636B002020202020204E6D415A2A
:1001B000740055702F446F776E202020205A75727E
:1001C000636B002020202020204E6D535A74004580
:1001D00072726F72005A7572636B0053746E64654D
:1001E000004D696E746500202020202020202020F2
:1001F0002020002020202020204E6D5A5A740045D7
:1002000072726F72005A7572636B0053746E64651C
:10021000004D696E746500202020202020202020C1
:100220002020002020202020204E6D415A740045BF
:1002300072726F72005A7572636B0053746E6465EC
:10024000004D696E74650020202020202020202091
:100250002020002020202020204E6D535A7400556D
:10026000702F446F776E202020205A7572636B00C8
:10027000204E6D566B7A00202020202020004572F1
:10028000726F720053746F7020005A7572636B0046
:100290005374617274004572726F720053764E75BA
:1002A0006C005376537274004572726F72005A7507
:1002B00072636B0053764E756C0053765372740004
:1002C0004E6D537672004572726F720053746F7088
:1002D00020005A7572636B005374617274002020A1
:1002E0002020202000204E6D5568720020005072A2
:1002F000536530005A7572636B0020202020202047
:100300000020507253653000202020202020202023
:1003100020200055702F446F776E202020205A75C2
:1003200072636B002053656B202020507250754221
:10033000000011241FBECFEFD4E0DEBFCDBF11E01F
:10034000A0E0B1E0E6E8FDE102C005900D92A23028
:10035000B107D9F711E0A2E0B1E001C01D92A332CC
:10036000B107E1F70E942C0E0C94C10E0C94000012
:10037000CF92DF92EF92FF920F931F93CF93DF9371
:10038000EC01488159816A817B81452B462B472BA3
:1003900071F10E94C102088119812A813B81601795
:1003A000710782079307A0F468017901C61AD70A7A
:1003B000E80AF90A8EEFC8168FEFD806E8068FE72D
:1003C000F806B8F0188219821A821B8280E012C0E7
:1003D0006B017C01C01AD10AE20AF30A8EEFC8163B
:1003E0008FEFD806E8068FE7F80660F302C08FEFBC
:1003F00001C081E0DF91CF911F910F91FF90EF90AD
:10040000DF90CF900895CF92DF92EF92FF92CF933B
:10041000DF93EC01411551056105710521F0415053
:100420005109610971096A017B018FEFC81AD80A65
:10043000E80AF80A8EEFC8168FEFD806E8068FE7AD
:10044000F80640F489EEC81683E0D806E104F1040A
:1004500068F007C08DEFC82EDD24DA94ED2C8FE70D
:10046000F82E8FEFC81AD80AE80AF80A0E94C102CB
:100470006C0D7D1D8E1D9F1D6115710581059105FA
:1004800029F0688379838A839B8308C041E050E028
:1004900060E070E0488359836A837B83DF91CF916A
:1004A000FF90EF90DF90CF900895CF92DF92EF9280
:1004B000FF920F931F93FC01009771F1C080D180D0
:1004C000E280F380C114D104E104F10429F18A012E
:1004D0009B010F5F1F4F2F4F3F4F0F3F8FEF1807AD
:1004E00028078FE33807C0F40C0D1D1D2E1D3F1D7E
:1004F000011511052105310529F00083118322839F
:10050000338308C041E050E060E070E040835183F5
:100510006283738380E001C08FEF1F910F91FF9082
:10052000EF90DF90CF900895FC011082118212822B
:1005300013820895CF93DF9300D000D0CDB7DEB7FC
:10054000AC0160E070E0CE0101960E940302CE0192
:1005500001960E94B8018111FACF0F900F900F9071
:100560000F90DF91CF91089584B5826084BD83E0C0
:1005700085BD89EF87BDEEE6F0E0808182608083F3
:1005800008952FB7F8946091020170910301809152
:100590000401909105012FBF08951F920F920FB68D
:1005A0000F9211242F933F934F935F936F937F93F9
:1005B0008F939F93AF93BF93CF93EF93FF938091CC
:1005C000020190910301A0910401B09105010196EF
:1005D000A11DB11D8093020190930301A09304011A
:1005E000B09305010E941304809101018150809312
:1005F0000101811112C0CAE0C09301010E941105DE
:100600000E941404809100018150809300018111A7
:1006100004C0C09300010E94D104FF91EF91CF91DB
:10062000BF91AF919F918F917F916F915F914F910A
:100630003F912F910F900FBE0F901F90189581152D
:10064000910511F00197F1F708959BB19F7087FD17
:10065000906886FD906485FD906284FD90619BB9F1
:100660005B9A5B989F7083FD906882FD906481FD2A
:10067000906280FD90619BB95B9A5B9880E892E004
:100680000C941F035A9881E00E94250380E190E4B6
:100690000C941F03CF93DF935A9AEC01899188231E
:1006A00019F00E942503FACFDF91CF910895CF93DF
:1006B000DF93EC015A9AFE018491882321F00E9475
:1006C00025032196F8CFDF91CF9108955A9A0C9483
:1006D00025035A98662349F0613011F4805C05C007
:1006E000623011F4805F01C0805B80680C94250348
:1006F0001F93CF93DF93D82F162FC42F0E94690327
:10070000CC2329F080E20E946603C150F9CF612F0B
:100710008D2FDF91CF911F910C946903FF920F935E
:100720001F93CF93DF93CDB7DEB72B970FB6F89417
:10073000DEBF0FBECDBF8C01F62E4BE050E060E275
:1007400070E0CE0101960E947E0E4AE050E0BE01AC
:100750006A5F7F4FC8010E94850EFC010190002056
:10076000E9F73197E81BF90B85E090E08F199109C3
:100770008E0F911D21E030E02C0F3D1F820F931F43
:100780000E944A032B960FB6F894DEBF0FBECDBF72
:10079000DF91CF911F910F91FF900895CF93C82FB4
:1007A000529A539A9AB1906F9AB95A985B9880E08E
:1007B0009AEF0E941F035C9A5D9A5B9A5B9880E2B5
:1007C0009EE40E941F035B9A5B9880E892E00E947F
:1007D0001F035B9A5B9880E892E00E941F035C987D
:1007E0005B9A5B9880E892E00E941F0388E20E9477
:1007F000250388E00E9425030E94420386E00E94B0
:10080000250386E00E9425038C2FCF910C942503AD
:1008100088B1807F88B987B18F6087B988B18960D6
:1008200088B9089508950895089508959FB7F89494
:1008300080930901882379F020910C0130910D01FA
:1008400030930F0120930E01833028F0809107012F
:100850008170809308019FBF08959FB7F89480919D
:1008600009019FBF08952FB7F89490930D018093CD
:100870000C012FBF08952FB7F89480910C0190912F
:100880000D012FBF08952FB7F89490930B0180931B
:100890000A012FBF08952FB7F89480910A01909113
:1008A0000B012FBF08959FB7F894809307019FBF56
:1008B00008959FB7F894809107019FBF08959FB74F
:1008C000F894809306019FBF08959FB7F894809194
:1008D00006019FBF089580910901882309F447C04C
:1008E00080910E0190910F01019790930F018093D9
:1008F0000E01892B51F480910C0190910D01909380
:100900000F0180930E014198429820910E01309181
:100910000F0180910A0190910B012817390709F006
:100920003FC080910801811105C081E080930801DA
:10093000429A03C010920801419A809109018330C4
:1009400078F1809107018F5F8C3318F48093070151
:1009500007C010920701809106018F5F8093060106
:10096000809106018831E0F01092060108954199C6
:1009700002C0429B15C080910E0190910F0101971A
:1009800090930F0180930E01892B51F480910C01FB
:1009900090910D0190930F0180930E014198429820
:1009A00008950C946B0485B18C6385B91092150180
:1009B000109214011092100110921701109216015A
:1009C0001092110110921901109218011092120147
:1009D00010921B0110921A011092130108959FB7F3
:1009E000F894E82FF0E0E05FFE4F80819FBF08950C
:1009F0002FB7F894E82FF0E0EE0FFF1FEC5EFE4FEC
:100A0000808191812FBF08959FB7F894E82FF0E07F
:100A1000E05FFE4F8081882311F0806880839FBF54
:100A200008951A9918C080911401909115010196AA
:100A300090931501809314018530910521F48091E4
:100A40001001816005C0C29761F48091100182603D
:100A50008093100106C0109215011092140110929B
:100A600010011B9918C080911601909117010196F1
:100A700090931701809316018530910521F48091A0
:100A80001101816005C0C29761F4809111018260FB
:100A90008093110106C01092170110921601109256
:100AA00011011C9918C080911801909119010196AB
:100AB00090931901809318018530910521F480915C
:100AC0001201816005C0C29761F4809112018260B9
:100AD0008093120106C01092190110921801109211
:100AE00012011D9918C080911A0190911B01019665
:100AF00090931B0180931A018530910521F4809118
:100B00001301816005C0C29761F480911301826076
:100B100080931301089510921B0110921A011092F4
:100B2000130108950E9408040E94D3040C949906AE
:100B30000E949D0680E00E94EF041816DCF780E01A
:100B40000E94040580E0089580E00E9416040E943F
:100B5000D4080E942F0780E00E94EF041816CCF7FB
:100B600080E00E940405F5CF08951F93CF93DF9393
:100B7000C82F162FD42F82E00E94EF0481FF09C0F6
:100B80008AEF90E00E949A02CF5FDC1740F4C12FF9
:100B900006C0181624F482E00E940405F5CF83E015
:100BA0000E94EF0481FF0AC08AEF90E00E949A023F
:100BB0008FEF8C0FD81740F48D2F0AC018163CF415
:100BC00083E00E940405F4CF8117B0F301C08C2F9D
:100BD000DF91CF911F910895CF93DF930E94140866
:100BE000D82FC1E0813009F4C0E06D2F8C2F0E9416
:100BF000B10641E060E08C2F0E94B505C82F80E06F
:100C00000E94EF0418168CF780E00E9404058C2FD8
:100C1000DF91CF910895CF93C0E08C2F0E94710790
:100C200047E060E08C2F0E94B505C82F80E00E944D
:100C3000EF04181694F780E00E940405C11103C068
:100C40000E945209EACFC13019F40E947B0BE5CF14
:100C5000C23019F40E94B209E0CFC33019F40E94E7
:100C6000D409DBCFC43019F40E94450AD6CFC53071
:100C700019F40E94B60AD1CFC63021F0C73069F608
:100C800082E001C081E0CF910895CF93C0E08C2F26
:100C90000E94040743E060E08C2F0E94B505C82F36
:100CA00080E00E94EF04181694F780E00E9404058B
:100CB000C11103C00E94980DEACFC13019F40E94FF
:100CC000BB0DE5CFC23021F0C33009F782E001C08F
:100CD00080E0CF910895CF93C0E08C2F0E94D4077D
:100CE00041E060E08C2F0E94B505C82F80E00E9493
:100CF000EF0418162CF480E00E9404058C2F09C024
:100D000081E00E94EF04181644F781E00E94040578
:100D100080E0CF910895CF93C82F0E94EF0418165A
:100D20002CF48C2F0E94040580E001C081E0CF915B
:100D300008958CE00C94CE03089560E080E00E945A
:100D400069038DE691E00E94570389E691E00E94D5
:100D5000570361E080E00E9469038CE591E00C9408
:100D60005703CF93DF93D82FC62F60E080E00E9417
:100D700069038BE491E00E94570361E080E00E94E8
:100D8000690389E491E00E945703C6FF03C087E42A
:100D900091E002C085E491E00E94570383E491E072
:100DA0000E94570381E491E00E9457038FE391E092
:100DB0000E945703C2FF03C08DE391E002C08BE3A2
:100DC00091E00E945703C1FF03C089E391E002C094
:100DD00087E391E00E945703C0FF03C085E391E0E1
:100DE00002C083E391E00E9457038FE291E00E94EA
:100DF0005703D11103C089E291E002C083E291E080
:100E0000DF91CF910C945703CF93C82F60E080E01F
:100E10000E9469038CEC90E00E94570361E080E03F
:100E20000E94690380EC90E00E945703C11103C047
:100E30008AEB90E011C0C13019F484EB90E00CC053
:100E4000C23019F48EEA90E007C0C33019F488EA82
:100E500090E002C082EA90E0CF910C94570360E0EA
:100E600080E00E9469038BE790E00E94570387E7C8
:100E700090E00E94570361E080E00E9469038CE6E5
:100E800090E00C945703CF93C62F90E062E08C590A
:100E90009F4F0E948E038AE690E00E9457038C2F9A
:100EA00090E062E08C599F4FCF910C948E03CF93CA
:100EB000DF93C82F6AE00E944A0ED82F62E090E0CC
:100EC0000E948E0388E690E00E9457038C2F9AE0E0
:100ED000D99F8019112461E090E0DF91CF910C94AB
:100EE0008E031F93CF93DF931F92CDB7DEB7182FDA
:100EF00060E080E00E9469030E943C0989830E94AF
:100F0000420969810E94430781E291E00E945703F0
:100F10000E9436090E9457078AE191E00E94570318
:100F200061E085E00E94690383E191E00E9457033C
:100F3000111103C08DE091E025C0113019F487E054
:100F400091E020C0123019F481E091E01BC0133011
:100F500019F48BEF90E016C0143019F485EF90E08F
:100F600011C0153019F48FEE90E00CC0163019F452
:100F700089EE90E007C0173019F483EE90E002C0CC
:100F80008DED90E00E94570361E080E00E946903CC
:100F90000E94590489830E94650469810F90DF9142
:100FA000CF911F910C9443071F93CF93DF931F9210
:100FB000CDB7DEB7182F60E080E00E9469030E9481
:100FC0003C0989830E94420969810E94430780EAA3
:100FD00090E00E9457030E9436090E94570789E952
:100FE00090E00E94570361E085E00E94690382E976
:100FF00090E00E945703111103C08CE890E002C0FA
:1010000086E890E00E94570361E080E00E94690357
:101010000E94590489830E94650469810F90DF91C1
:10102000CF911F910C944307CF9380E090E00E94F2
:101030009B0E80931C018A3F08F461C010921C0132
:1010400081E08093220184E68093210110922001A7
:1010500010921F0110921E0110921D018CE390E06E
:101060000E9433048AE090E00E94430480E00E94E2
:10107000530487E10E945F0460911C0180E090E0CE
:101080000E94A30E6091220189E090E00E94A30ECD
:101090006091210188E090E00E94A30E6091200100
:1010A00084E090E00E94A30E60911F0183E090E035
:1010B0000E94A30E60911E0182E090E00E94A30EA8
:1010C00060911D0181E090E00E94A30E0E944B04FC
:1010D000682F87E090E00E94A30E0E945904682FB9
:1010E00086E090E00E94A30E0E946504682F85E0D0
:1010F00090E00E94A30E80912201846046C089E0A6
:1011000090E00E949B0E8093220188E090E00E9474
:101110009B0EC82F8093210184E090E00E949B0EDB
:101120008093200183E090E00E949B0E80931F013A
:1011300082E090E00E949B0E80931E0181E090E08F
:101140000E949B0E80931D016C2F70E080E797E159
:101150000E94560ECB010E94330487E090E00E946B
:101160009B0E90E00E94430486E090E00E949B0E5C
:101170000E94530485E090E00E949B0E0E945F0451
:1011800080912201882321F082608093220108C08F
:1011900081E08093220161E089E090E00E94A30E4B
:1011A00080912201CF9108958091220180748093D3
:1011B000220160911C0180E090E00E94A30E6091EA
:1011C000220189E090E00E94A30E6091210188E055
:1011D00090E00E94A30E6091200184E090E00E94C4
:1011E000A30E60911F0183E090E00E94A30E609126
:1011F0001E0182E090E00E94A30E60911D0181E03B
:1012000090E00E94A30E0E944B04682F87E090E0BC
:101210000E94A30E0E945904682F86E090E00E946D
:10122000A30E0E946504682F85E090E00C94A30E45
:1012300080932201089580912201089580931C01DA
:10124000089580911C0108958A3028F0682F88370E
:1012500018F067E701C06AE06093210170E080E761
:1012600097E10E94560ECB010C943304809121012A
:10127000089580932001089580912001089580931E
:101280001F01089580911F01089580931E01089504
:1012900080911E01089580931D01089580911D0184
:1012A00008950895CF93DF93C0E08C2F0E94B20B76
:1012B00041E060E08C2F0E94B505C82F80E00E94BD
:1012C000EF0418160CF040C080E00E940405C11124
:1012D00046C083E00E94160482E00E94B20B0E9486
:1012E0006504D82F0E944E09D81307C00E945904E4
:1012F000D82F0E944809D81741F080E00E94EF04DF
:1013000018163CF480E00E94040580E00E94160458
:101310001BC082E00E94EF04181644F482E00E9491
:1013200004050E9436098F5F0E94240983E00E9411
:10133000EF0418168CF683E00E9404050E9436091B
:1013400081500E942409C8CF81E00E94EF04181642
:101350000CF0ABCF81E0DF91CF910C940405DF91CD
:10136000CF910895CF930E943609C82F8C2F0E94E9
:101370008E0C47E76AE08C2F0E94B505C82F80E0ED
:101380000E94EF0418163CF480E00E9404058C2FA4
:10139000CF910C94240981E00E94EF04181634F7D1
:1013A00081E0CF910C9404051F93CF93DF93C0E0AD
:1013B0008C2F0E94A80C42E060E08C2F0E94B505A3
:1013C000C82F80E00E94EF0418160CF04EC080E099
:1013D0000E940405C11125C00E943C09D82F0E941B
:1013E0004209182F612F8D2F0E944A0D4BE360E0B8
:1013F0008D2F0E94B505D82F80E00E94EF041816AB
:101400003CF480E00E9404058D2F0E9439092DC014
:1014100081E00E94EF0418162CF781E00E94040579
:1014200024C0C13071F50E943C09182F0E94420966
:10143000D82F6D2F812F0E944A0D47E160E08D2F3C
:101440000E94B505D82F80E00E94EF0418163CF4E6
:1014500080E00E9404058D2F0E943F0906C081E0B4
:101460000E94EF0418162CF7D8CF81E00E94EF04F9
:1014700018160CF09DCF81E0DF91CF911F910C9455
:101480000405DF91CF911F9108951F93CF93DF93B0
:10149000C0E08C2F0E94DE0C42E060E08C2F0E94A6
:1014A000B505C82F80E00E94EF0418160CF04EC05E
:1014B00080E00E940405C11125C00E945904D82F64
:1014C0000E946504182F612F8D2F0E94640D4BE33D
:1014D00060E08D2F0E94B505D82F80E00E94EF04B8
:1014E00018163CF480E00E9404058D2F0E945304DE
:1014F0002DC081E00E94EF0418162CF781E00E94B5
:10150000040524C0C13071F50E945904182F0E94AF
:101510006504D82F6D2F812F0E94640D47E160E094
:101520008D2F0E94B505D82F80E00E94EF04181679
:101530003CF480E00E9404058D2F0E945F0406C0E9
:1015400081E00E94EF0418162CF7D8CF81E00E94AA
:10155000EF0418160CF09DCF81E0DF91CF911F9121
:101560000C940405DF91CF911F9108951F93CF93A1
:10157000DF93C0E08C2F0E94140D42E060E08C2FBE
:101580000E94B505C82F80E00E94EF0418160CF0E9
:101590004EC080E00E940405C11125C00E94480988
:1015A000D82F0E944E09182F612F8D2F0E947E0D7B
:1015B0004BE360E08D2F0E94B505D82F80E00E949C
:1015C000EF0418163CF480E00E9404058D2F0E9461
:1015D00045092DC081E00E94EF0418162CF781E028
:1015E0000E94040524C0C13071F50E944809182FDB
:1015F0000E944E09D82F6D2F812F0E947E0D47E14A
:1016000060E08D2F0E94B505D82F80E00E94EF0486
:1016100018163CF480E00E9404058D2F0E944B09AF
:1016200006C081E00E94EF0418162CF7D8CF81E0A5
:101630000E94EF0418160CF09DCF81E0DF91CF914E
:101640001F910C940405DF91CF911F9108950F9382
:101650001F93CF93DF93082F811107C00E943C098D
:10166000182F0E944209D82F02C0D0E010E0C0E03D
:101670002D2F412F6C2F802F0E943E0C41E060E007
:101680008C2F0E94B505C82F80E00E94EF04181629
:101690000CF580E00E940405C11128C083E00E947F
:1016A00016042D2F412F62E0802F0E943E0C0E94D5
:1016B00065048D1304C00E945904811741F080E035
:1016C0000E94EF0418166CF780E00E94040580E089
:1016D0000E94160481E00E94EF0418164CF681E087
:1016E000DF91CF911F910F910C940405DF91CF9161
:1016F0001F910F9108951F93CF93DF930E94420390
:1017000010E0812F0E94FC0B42E060E0812F0E94DC
:10171000B505182F80E00E94EF04181694F480E0BD
:101720000E9404051230C0F40E943B04EC018AE0E0
:1017300090E00E943304812F0E94270BCE010E946B
:10174000330481E00E94EF041816DCF681E0DF919B
:10175000CF911F910C940405DF91CF911F910895B3
:10176000089508951F93CF93DF931F92CDB7DEB7EF
:10177000182F60E080E00E9469030E943C09898381
:101780000E94420969810E9443078CEE92E00E9408
:1017900057030E9436090E94570785EE92E00E9487
:1017A000570361E085E00E9469038EED92E00E949C
:1017B0005703111103C088ED92E00CC0113019F4E9
:1017C00082ED92E007C0123019F48CEC92E002C076
:1017D00086EC92E00E94570361E080E00E9469037A
:1017E0000E94590489830E94650469810F90DF91EA
:1017F000CF911F910C9443071F93CF93DF931F92B8
:10180000CDB7DEB7182F60E080E00E9469030E9428
:101810003C0989830E94420969810E94430760E074
:101820008BE00E94690380EC92E00E94570361E024
:1018300080E00E9469030E94590489830E94650424
:1018400069810E94430761E08BE00E9469031111E6
:1018500003C08AEB92E00CC0113019F484EB92E0E3
:1018600007C0123019F48EEA92E002C088EA92E0D2
:101870000F90DF91CF911F910C9457030F931F93FB
:10188000CF93DF9300D0CDB7DEB7082F162F60E0DF
:1018900080E02A8349830E9469034981642F2A8159
:1018A000822F0E94430760E08BE00E9469030111D0
:1018B00003C082EA92E007C0013019F48CE992E09B
:1018C00002C086E992E00E94570361E080E00E9436
:1018D00069030E94590489830E94650469810E94FA
:1018E000430761E08BE00E946903111103C080E9A6
:1018F00092E00CC0113019F48AE892E007C012306F
:1019000019F484E892E002C08EE792E00F900F9005
:10191000DF91CF911F910F910C945703CF93C82F54
:1019200060E080E00E94690387E792E00E9457032D
:101930008C2F0E94570780E792E00E94570361E0D6
:1019400080E00E9469038FE592E0CF910C945703E9
:101950001F93CF93DF931F92CDB7DEB7182F60E0B0
:1019600080E00E9469030E943C0989830E94420929
:1019700069810E94430783E592E00E94570361E07A
:1019800080E00E94690387E492E00E9457031111EE
:1019900003C081E492E00CC0113019F48BE392E0B3
:1019A00007C0123019F485E392E002C08FE292E0A2
:1019B0000F90DF91CF911F910C9457031F93CF93FA
:1019C000DF931F92CDB7DEB7182F60E080E00E9452
:1019D00069030E94590489830E94650469810E94F9
:1019E000430783E292E00E94570361E080E00E9497
:1019F000690387E192E00E945703111103C081E15E
:101A000092E00CC0113019F48BE092E007C0123064
:101A100019F485E092E002C08FEF91E00F90DF9122
:101A2000CF911F910C9457031F93CF93DF931F9275
:101A3000CDB7DEB7182F60E080E00E9469030E94F6
:101A4000480989830E944E0969810E94430783EFF8
:101A500091E00E94570361E080E00E94690387EEF5
:101A600091E00E945703111103C081EE91E00CC078
:101A7000113019F48BED91E007C0123019F485EDA7
:101A800091E002C08FEC91E00F90DF91CF911F9118
:101A90000C945703CF93DF93D82FC62F60E080E0DC
:101AA0000E9469036D2F8C2F0E94430783EC91E005
:101AB0000E94570361E080E00E94690382EB91E09D
:101AC000DF91CF910C945703CF93DF93D82FC62F7C
:101AD00060E080E00E9469036D2F8C2F0E94430715
:101AE00086EA91E00E94570361E080E00E9469036A
:101AF00085E991E0DF91CF910C945703CF93DF9369
:101B0000D82FC62F60E080E00E9469036D2F8C2FD4
:101B10000E94430789E891E00E94570361E080E05A
:101B20000E94690388E791E0DF91CF910C945703FD
:101B3000CF930E944B04C82F8C2F0E94E20D43E1EB
:101B400065E08C2F0E94B505C82F80E00E94EF044D
:101B5000181644F480E00E9404058C2F90E0CF9189
:101B60000C94430481E00E94EF0418162CF781E0E6
:101B7000CF910C940405CF93C0E08C2F0E94F80DF8
:101B800041E060E08C2F0E94B505C82F80E00E94E4
:101B9000EF04181664F480E00E940405C13081F45B
:101BA00080E00E94530480E0CF910C945F0481E0B8
:101BB0000E94EF0418160CF781E0CF910C940405F5
:101BC000CF910895CF93C82F60E080E00E94690311
:101BD0008C2F0E94570784E293E00E94570361E034
:101BE00080E00E94690383E193E0CF910C94570356
:101BF0001F93CF93DF931F92CDB7DEB7182F60E00E
:101C000080E00E94690388E093E00E94570381E02E
:101C100093E00E94570361E085E00E9469038AEF28
:101C200092E00E945703111103C084EF92E002C0BA
:101C30008EEE92E00E94570361E080E00E9469030B
:101C40000E94590489830E94650469810F90DF9185
:101C5000CF911F910C944307CF930E9492050E944D
:101C6000B40278940E9498050E94EC05C82FC130F8
:101C700011F40E9445060E940B06C82F8230B8F36B
:101C80000E946B06882399F30E94A40580E090E0EF
:101C9000CF910895991B79E004C0991F961708F019
:101CA000961B881F7A95C9F78095089597FB072E94
:101CB00016F4009407D077FD09D00E946A0E07FC45
:101CC00005D03EF4909581959F4F0895709561954C
:101CD0007F4F0895AA1BBB1B51E107C0AA1FBB1F62
:101CE000A617B70710F0A61BB70B881F991F5A95A8
:101CF000A9F780959095BC01CD010895DC0101C044
:101D00006D9341505040E0F70895FB019F01423030
:101D100074F0453264F4642F77270E946A0E805D68
:101D20008A330CF0895D8193CB010097A1F7108273
:101D3000C9010C94B10EF999FECF92BD81BDF89AFC
:101D4000992780B50895262FF999FECF1FBA92BD25
:101D500081BD20BD0FB6F894FA9AF99A0FBE01968C
:101D60000895DC01FC01672F71917723E1F7329729
:101D700004C07C916D9370836291AE17BF07C8F366
:061D80000895F894FFCF66
:021D86000A0A47
:00000001FF
